:100000000C941E060C94B8270C94E5270C94460615
:100010000C94E8120C9446060C9446060C94460682
:100020000C9446060C9446060C9446060C94460620
:100030000C9446060C9446060C9446060C94460610
:100040000C9412280C9446060C94E32B0C94262C4A
:100050000C9446060C9446060C9446060C944606F0
:100060000C9446060C9446064818AA1889188C1851
:100070008F189218951898189B18AA18A418DC19AC
:10008000DE19DE19DC19DE19DE19DE19DE19DE19BA
:10009000DE19DE19DE19DE19DE19DE19DE19DE19A8
:1000A0006219DE19DE19DE19DE19DE19D318DE1920
:1000B000DE19DE19DE19DE19DE19DE19DE19DE1988
:1000C000DE19DE19DE19DE19DE19DE196E196E1958
:1000D0006E196E196E196E196E196E196E19DE1978
:1000E000DE19DE19DE19DE19DE19D3186D196D1946
:1000F0006D196D19DE197B19811987198D199319DD
:1001000099199F19A519AF19B919C319CD1914193E
:10011000D618DE19DE19DE19DE196219DE19DE19AC
:10012000DE19DE19DE19DE19DE19DE196C196C19FB
:100130006C196C19DE197B19811987198D1993199E
:1001400099199F19A519AF19B919C319CD191419FE
:10015000D618DE19DE19DE19DE196219111A111A04
:10016000111A111A111A111A111A111A111A111A37
:10017000111A111A111A281B281B281B281B281BAF
:10018000281B561A601A6A1A741AD21ADC1AEB1A49
:10019000FC1A841C991CA51CAE1CBD1CE21CEB1C8B
:1001A000341DFD1C47204D2053205A2068208A20F2
:1001B000A820456E746572206D656E752E2E2E001A
:1001C000546F67676C6564206D6963726F50504D42
:1001D00000546F67676C656420696E76657274653C
:1001E000642050504D2100546F67676C6564205443
:1001F00058206D7574696E672100546F67676C6570
:10020000642074656C656D65747279210050726F3D
:10021000746F636F6C206572726F72207769746897
:100220002052580054696D656F7574207768656E4B
:1002300020636F6E6E656374696E6720746F205201
:100240005800507265737320616E79206B65792058
:10025000746F2063616E63656C00436F6E6E6563DF
:1002600074696E6720746F2052582C20706F776508
:100270007220757020746865205258202877697440
:10028000682062696E6420706C7567206966206EF4
:100290006F74207573696E6720616C776179732064
:1002A00062696E642900546F67676C656420276912
:1002B0006D6D656469617465206F75747075742700
:1002C00000546F67676C65642027736C61766520E6
:1002D0006D6F64652700546F67676C6564202761E4
:1002E0006C776179732062696E642700546F676769
:1002F0006C65642050504D206368616E6E656C20A3
:100300006C696D69740053657420525353492069B8
:100310006E6A656374696F6E206368616E6E656C8A
:100320002028303D3D64697361626C652900536526
:10033000742050504D206D696E696D756D20737914
:100340006E630053657420626561636F6E20696E31
:1003500074657276616C0053657420626561636FC9
:100360006E2064656C617900536574206265616319
:100370006F6E206672657175656E637920696E2097
:10038000487A3A20303D64697361626C652C205074
:10039000783D504D52206368616E6E656C20782CFC
:1003A0002046783D465253206368616E6E656C202E
:1003B00078005365742050574D2073746F7020641B
:1003C000656C61792028302064697361626C6564B2
:1003D0002C20312D323535203D3D20302E317320FB
:1003E0002D2035306D696E29005365742050504DB5
:1003F0002073746F702064656C61792028302064EC
:10040000697361626C65642C20312D323535203D75
:100410003D20302E3173202D2035306D696E29003E
:10042000536574206661696C736166652064656CF0
:1004300061792028302064697361626C65642C20C6
:10044000312D323535203D3D20302E3173202D2089
:1004500035306D696E29002A2A2A2A2A2A2A2A2A50
:100460002A2A2A2A2A2A2A2A2A2A2A2A2A2A2A2AEC
:100470002A2A2A2A0052582041636B6564202D20C5
:1004800072657665727420737563636573736675E0
:100490006C21002A2A2A2A2A2A2A2A2A2A2A2A2AAD
:1004A0002A2A2A2A2A2A2A2A2A2A2A2A2A2A2A2AAC
:1004B000002A2A2A2A2A2A2A2A2A2A2A2A2A2A2AC6
:1004C0002A2A2A2A2A2A2A2A2A2A2A2A2A2A00528E
:1004D000582041636B6564202D20757064617465DC
:1004E000207375636365737366756C21002A2A2A0D
:1004F0002A2A2A2A2A2A2A2A2A2A2A2A2A2A2A2A5C
:100500002A2A2A2A2A2A2A2A2A2A0056616C696457
:100510002063686F69636573206172653A205B319F
:100520005D2D5B31365D20286368616E6E656C20E1
:10053000312D31362900536574206F7574707574D0
:1005400020666F7220706F727420005B585D2061AE
:10055000626F7274206368616E67657320616E6498
:10056000206578697420525820636F6E6669670051
:100570005B535D20736176652073657474696E6783
:100580007320746F205258005B525D20726576654F
:1005900072742052582073657474696E6773207486
:1005A0006F2064656661756C747300557365206EA9
:1005B000756D62657273205B312D445D20746F2010
:1005C0006564697420706F727473205B452D515D92
:1005D00020666F722073657474696E677300202DD6
:1005E00020726563656976657220636F6E66696700
:1005F000757261746F722C20727820737720000AF4
:100600000A6F70656E4C52536E67200053657420FC
:1006100073657269616C2062617564726174653AB8
:10062000200056616C69642063686F696365733A82
:100630002031202D20342B34202F2032202D203823
:10064000202F2033202D20382B34202F2034202D14
:10065000203132202F2035202D2031322B34202FF5
:100660002036202D20313600536574204368616E9A
:100670006E656C20636F6E6669673A20005365741F
:100680002044617461726174652028302D32293AEA
:10069000200053657420486F70206368616E6E653A
:1006A0006C7320286D61782032342C207365706162
:1006B000726174656420627920636F6D6D61732966
:1006C0002076616C69642076616C75657320312DCC
:1006D0003235353A2000536574206368616E6E656B
:1006E0006C2073706163696E6720287831306B48C5
:1006F0007A293A200053657420524620706F77653E
:10070000722028302D37293A200053657420524634
:10071000206D6167696320286865782920652E67E8
:100720002E20307844454144463030443A2000532E
:1007300065742062617365206672657175656E63AC
:10074000792028696E20487A293A20005B5A5D207A
:10075000656E746572207265636569766572206383
:100760006F6E66696775726174696F6E2075746902
:100770006C79005B465D20646973706C61792061FF
:10078000637475616C206672657175656E63696509
:10079000732075736564005B525D2063616C6375E3
:1007A0006C6174652072616E646F6D206B65792079
:1007B000616E6420686F70206C697374005B495DC2
:1007C000207265696E697469616C697A6520736508
:1007D0007474696E677320746F20736B65746368DB
:1007E0002064656661756C7473005B585D2072658A
:1007F00076657274206368616E67657320616E64EC
:100800002065786974206D656E75005B535D20739B
:100810006176652073657474696E677320746F20E8
:10082000454550524F4D20616E64206578697420B3
:100830006D656E7500557365206E756D62657273BA
:10084000205B302D395D20746F20656469742070E1
:100850006172616D657465727300202D2053797328
:1008600074656D20636F6E66696775726174696F18
:100870006E000A0A6F70656E4C52536E672000510D
:1008800029204F7574707574206265666F726520DB
:100890006C696E6B20283D465329203A2000502970
:1008A00020536C617665206D6F64652028657870D3
:1008B0006572696D656E74616C293A20004F29205C
:1008C00054696D65642042494E44206174207374FC
:1008D000617274757020203A20004E292050504DCE
:1008E000206F7574707574206C696D69746564200F
:1008F000202020203A200044495341424C454400E6
:100900004D292050504D205253534920746F20637D
:1009100068616E6E656C202020203A20004C2920F2
:1009200050504D206D696E696D756D2073796E63E1
:10093000202875732920203A200044495341424C15
:100940004544004B29204661696C736166652062ED
:100950006561636F6E20696E74762E2028312D32AA
:10096000353573293A20004A29204661696C736144
:10097000666520626561636F6E2064656C617920D5
:1009800028302D323535203D3E20313073202D204A
:100990003135306D696E293A200049292046616958
:1009A0006C7361666520626561636F6E206672714B
:1009B0002E203A200048292050574D2073746F7024
:1009C0002064656C6179202020202020203A2000BE
:1009D00047292050504D2073746F702064656C61FE
:1009E00079202020202020203A200046292046611E
:1009F000696C736166652064656C617920202020D4
:100A00002020203A200050574D206368616E6E65AB
:100A10006C200066756E6374696F6E3A2000292041
:100A2000706F72742000506F776572546F776572C3
:100A300000445446205548462033322D62697420C4
:100A400031306368004F70656E4C52536E67525878
:100A5000206D696E6920342F36636800466C7974A6
:100A6000726F6E2F4F72616E6765525820554846FF
:100A70002038636800525820747970653A20004429
:100A8000697361626C656400487A00203D3D200016
:100A900043616C63756C61746564207061636B6540
:100AA0007420696E74657276616C3A200042292068
:100AB0004D6963726F202868616C66292050504D23
:100AC000202020203A00412920496E766572746505
:100AD000642050504D20696E20202020203A0030A4
:100AE00029204D7574652062757A7A657220286DAB
:100AF0006F73746C79293A003929205365726961E2
:100B00006C2062617564726174653A00736D617224
:100B100074506F7274004672536B79005472616E38
:100B200073706172656E740044697361626C6564B0
:100B30000038292054656C656D657472793A2020FF
:100B40002020202020003729204368616E6E656CCC
:100B500020636F6E6669673A202000362920446161
:100B60007461726174652028302D32293A2020206A
:100B700000352920486F70206368616E6E656C7364
:100B80003A2020202020003429204368616E6E65C1
:100B90006C2073706163696E673A202000332920EE
:100BA000524620706F7765722028302D37293A2001
:100BB0002020003229205246206D616769633A2067
:100BC0002020202020202020003129204261736530
:100BD000206672657175656E63793A202020000089
:100BE00000000700020100000304060000000000EE
:100BF00000000001020408102040800102040810D7
:100C00002001020408102004040404040404040263
:100C10000202020202030303030303000000002395
:100C2000002600290000000000250028002B0000FD
:100C3000000000240027002A0000142D11241FBEEC
:100C4000CFEFD8E0DEBFCDBF13E0A0E0B1E0E6E338
:100C5000F0E602C005900D92A83CB107D9F716E066
:100C6000A8ECB3E001C01D92AC38B107E1F71CE07D
:100C7000CCE3DCE004C02297FE010E941D2ECA33A3
:100C8000D107C9F70E94502D0C9419300C94000024
:100C900080917105813019F482E080937105809113
:100CA0007105833019F484E0809371050895A89547
:100CB0000895DC01ED91FC910190F081E02D099502
:100CC00008952091720530917305382748E0C901D5
:100CD000880F991F37FF06C09C0151E2252750E17C
:100CE000352701C09C01415091F730937305209343
:100CF0007205089588E38093740580E092ECA1E08A
:100D0000B0E08093750590937605A0937705B09336
:100D1000780587E08093810580EC9AECA9E8B6E33A
:100D20008093790590937A05A0937B05B0937C0519
:100D300085E0809382058DEE9EEFADEABEED809357
:100D40007D0590937E05A0937F05B0938005E3E831
:100D5000F5E080E090E0863028F4DC01AF54BC4F31
:100D60002C9101C020E0219301968831910599F7DB
:100D700082E080939B058AE080939C05089580EC37
:100D800097EFAAEBB7E38093B9059093BA05A093C8
:100D9000BB05B093BC0580E090E0A0E0B0E5809397
:100DA000BD059093BE05A093BF05B093C005E1ECCF
:100DB000F5E080E081938F5F8031E1F70895A0E056
:100DC000B0E0E5EEF6E00C94E62DD82F0E946828FE
:100DD0006115710581059105C9F30E94892E109254
:100DE0007D0510927E0510927F0510928005C4E06B
:100DF000812C912C54018A94C0907D05D0907E0561
:100E0000E0907F05F0908005FE2CED2CDC2CCC24AE
:100E10000E94842EA50194010E94C52D6C0D7D1D9C
:100E20008E1D9F1D60937D0570937E0580937F05C9
:100E300090938005C15001F7DD2309F450C003E809
:100E400015E0E801A12CB12C62E3C62ED12CE12CD7
:100E5000F12C8881882309F442C0B39419F40E94CC
:100E60007A063DC00E94842EA70196010E94C52DDE
:100E7000E1E0E60FA3E8B5E08A2F801B8A1520F495
:100E80008D918E13F9CFE9CF2091820530E0A0E15A
:100E9000B7E20E945D2D9B01AC01AE2FB0E00E9435
:100EA0006C2D4090790550907A0560907B0570908C
:100EB0007C05640D751D861D971D4090B9055090E9
:100EC000BA056090BB057090BC05461657066806CB
:100ED000790618F2E993A39488E1A812BACFCDB7A6
:100EE000DEB7E0E10C94022E8436910520F4BC01BB
:100EF00080E090E017C09C018E3B910528F42A55B4
:100F00003109AAE0B0E00CC0823D910528F4245BD1
:100F10003109A4E6B0E004C02D5C3109A8E5B2E0D7
:100F20000E945D2DA4E6B0E09B01AC010E946C2DF7
:100F3000089590E08C599F4F0E947407089561E0D6
:100F400089E00E94152960E089E00E944E290895F9
:100F5000892B11F061E001C060E089E00E944E2918
:100F6000089560E08EE00E94152961E08FE00E9404
:100F7000152961E082E00E94152960E083E00E946B
:100F8000152961E084E00E941529089542E050E0AF
:100F900068E476E081E00E9498270895E3E0F0E0BD
:100FA00089E080935700E491E67081E0E63009F033
:100FB00080E00895CF93DF93C82F0E94CE07882347
:100FC00081F0DFB781E080937005F8940E945706A6
:100FD00088E180936000C0936000C1110E945706B1
:100FE000DFBFDF91CF9108958F929F92AF92BF9212
:100FF000CF92DF92EF92FF92CF93FC01C0A5EC2F2E
:10100000E770F0E0E758FC4FA081B0E0C7FF03C0F5
:1010100024E130E002C02FE030E0FC0197A183E141
:10102000989FF0011124E25CFE4F80809180A280A5
:10103000B380A20FB31F20E43FE14DE750E00E94D0
:10104000772DA50194010E94A32D8C2F887149F45E
:1010500069017A01E0EDCE0EE7E0DE1EE11CF11C35
:101060001BC0C7FF05C060E47AE88CE29EE004C0C4
:1010700060E07EEE8AEB9BE069017A01F8EBCF0E2F
:10108000FBE0DF1EE11CF11CA50194010E94A32DD1
:10109000C20ED31EE41EF51EC701B60169517C4F76
:1010A0008F4F9F4F28EE33E040E050E00E94A32D89
:1010B000A8EEB3E00E946C2DCF91FF90EF90DF90EF
:1010C000CF90BF90AF909F908F9008958F3F9105E4
:1010D00051F048F0811522E0920738F081159340D5
:1010E00030F482E0089580E0089581E0089583E07F
:1010F0000895A0E0B0E0EFE7F8E00C94EF2DEB01ED
:101100008A01B82FB695A0E028813981F8012083A3
:101110002A813B8121832C813D8122832E813F8145
:101120002383688179814A815B812C813D81EE81B5
:10113000FF819F2F9295990F990F907C272F2370F5
:10114000922B252F2370220F220F922B232F2370F7
:101150002295207F922BF80194830B5F1F4F2896D6
:10116000AF5FBA1788F680FF24C0888199810E94FA
:101170006608D82E8A819B810E946608E82E8C81A1
:101180009D810E946608F82E8E819F810E946608CC
:10119000F0E4DF9EA001112490E1E99E900111246A
:1011A000242B282BE4E0FE9EB0011124262BF8010D
:1011B0002083CDB7DEB7E7E00C940B2E803223E01E
:1011C000920708F1883E23E0920740F48F51934044
:1011D000E4E096958795EA95E1F70895803D27E04C
:1011E000920718F48C5D93400895883928E092079F
:1011F00068F4885C974074E0969587957A95E1F756
:101200008D509C4F089580E090E008958FEF93E01B
:1012100008958C30910540F4A4E0880F991FAA9599
:10122000E1F7885D9C4F0895843F23E0920718F40E
:1012300084529C4F0895811524E0920740F486570C
:10124000934FF4E0880F991FFA95E1F7089580E92C
:1012500098E008959C013695279525753575821B74
:10126000930B9C0123733373969587959695879579
:1012700083739373820F931F9C0154E036952795D7
:101280005A95E1F7280F391F2F703F7041E051E068
:10129000249FC001259F900D349F900D1124892F0C
:1012A00008955A98882319F00000419A02C000005E
:1012B000419800005A9A000008955A9A000086B199
:1012C0005A98000081700895CF93DF93D82F5C9ACD
:1012D0005A985C98C8E08D2F80780E945109DD0FE4
:1012E000C150C9F75A98DF91CF9108958F770E9426
:1012F00064090895CF93DF93D82FC8E08D2F8078AD
:101300000E945109DD0FC150C9F75A98DF91CF9162
:101310000895CF93DF935A98C8E080E0D82FDD0F6F
:101320000E945D098D0FC150C9F7DF91CF910895DB
:101330000E9476090E9489095C9A0895A1E0B0E0B4
:10134000E4EAF9E00C94F42D806869830E94640952
:101350006981862F0E947A095C9A2196E2E00C94BA
:10136000102ECF93C0917D05C827E82FF0E0EC58F0
:10137000FA4F678589E70E949E096C2F8DE30E94D2
:101380009E096C2F82E40E949E09CF91089586E207
:101390000E9498090895CF93DF93EC016C818CE152
:1013A0000E949E096D818DE10E949E096E818EE1F1
:1013B0000E949E096F8180E20E949E09688581E2F9
:1013C0000E949E09698582E20E949E096A8583E2E5
:1013D0000E949E096B8584E20E949E096C8585E2CD
:1013E0000E949E096D858AE20E949E096E858EE6A6
:1013F0000E949E096F858FE60E949E09688980E79A
:101400000E949E09698981E70E949E096A8982E794
:101410000E949E09DF91CF910895CF92DF92EF92C3
:10142000FF92CF93DF936B017C01C11488E3D80650
:101430008CE9E8068CE1F80628F5C701B60120E83A
:1014400036E948E950E00E94A32DE901689760E879
:1014500079E687E69FEF0E947F2D6C0D7D1D8E1D26
:101460009F1DF2E0660F771F881F991FFA95D1F72D
:1014700021E732E040E050E00E94A32DF22EE32E5F
:1014800080E421C0C701B60120E03DE241E351E024
:101490000E94A32DE901689760E073ED8EEC9EEF4A
:1014A0000E947F2D6C0D7D1D8E1D9F1D660F771F69
:1014B000881F991F21E732E040E050E00E94A32DF1
:1014C000F22EE32E80E66C2F6F71680F85E70E9485
:1014D0009E096E2D86E70E949E096F2D87E70E9468
:1014E0009E09DF91CF91FF90EF90DF90CF9008950C
:1014F000682F8DE60E949E0908958F929F92AF9269
:10150000BF92CF92DF92EF92FF92CF93DF93D82FCB
:1015100083E00E94980980936F0584E00E949809F7
:1015200080936E0560E086E00E949E0961E087E09E
:101530000E949E096FE789E00E949E0965E08AE0AB
:101540000E949E0962E18BE00E949E0965E18CE0A9
:101550000E949E096DEF8DE00E949E0960E08EE082
:101560000E949E09DD2319F08BE291E008C02091D2
:101570009B0533E1239FC0011124825C9E4F0E9492
:10158000CB096CE880E30E949E096FE082E30E9431
:101590009E0962E483E30E949E0980919C0587FF77
:1015A00002C064E101C06AE084E30E949E096AE22D
:1015B00085E30E949E096DE286E30E949E0964ED28
:1015C00087E30E949E0960E088E30E949E0960E034
:1015D00089E30E949E09D11109C0C0907D05D09079
:1015E0007E05E0907F05F090800507C0C5E9CC2E10
:1015F000C1ECDC2EED2CCEEDFC2ECAE38F2C992411
:10160000AA24BB24682D8C2F0E949E09682D85E09A
:101610008C0F0E949E09FE2CED2CDC2CCC24CF5F7D
:10162000CE3361F76FEF83E40E949E096FEF84E48D
:101630000E949E096FEF85E40E949E096FEF86E489
:101640000E949E09DD2311F066E002C060918105D1
:101650008DE60E949E0960E089E70E949E096091E4
:1016600082058AE70E949E0960E083E70E949E0946
:1016700060E084E70E949E09D11109C0609179055C
:1016800070917A0580917B0590917C0504C060EC97
:101690007AEC89E896E30E940D0ADF91CF91FF90E2
:1016A000EF90DF90CF90BF90AF909F908F90089574
:1016B00061E087E00E949E0964E28EE70E949E0935
:1016C00063E088E00E949E0960E088E00E949E0935
:1016D00065E087E00E949E0962E085E00E949E0925
:1016E00083E00E94980980936F0584E00E94980926
:1016F00080936E05089583E00E94980980936F059A
:1017000084E00E94980980936E0561E087E00E9462
:101710009E096AE070E080E090E00E948B280E94C1
:10172000580B00000895CF92DF92FF920F931F9302
:10173000CF93DF931F92CDB7DEB7082F162F8EE31E
:1017400099830E949E09F02EC02E9981D92E8C2D4E
:101750008F19811738F4F60161916F018FE70E94AC
:101760009E09F5CF64E085E00E949E0983E00E9417
:10177000980980936F0584E00E94980980936E0514
:101780000E94682860936A0570936B0580936C05CE
:1017900090936D0569E087E00E949E0981E0809347
:1017A00071050F90DF91CF911F910F91FF90DF9006
:1017B000CF9008950F931F930E94930B8091710512
:1017C000813099F40E94682800916A0510916B0598
:1017D00020916C0530916D05601B710B820B930B92
:1017E000603A76488140910548F3809171058130D7
:1017F00031F46DE971E080EE95E00E94372A1F9187
:101800000F9108950F931F9380917105823021F4F9
:101810001092710581E020C0809171058130D9F46A
:101820000E94682800916A0510916B0520916C0553
:1018300030916D05601B710B820B930B613A7648FA
:101840008140910540F061E087E00E949E0910927E
:10185000710582E001C080E01F910F910895CF9340
:10186000DF93EC014AE050E06D2F70E080EE95E0F0
:101870000E94052B6EE280EE95E00E94092ABE01CF
:1018800084E0769567958A95E1F76F7077274AE04F
:1018900050E080EE95E00E94052B6EE280EE95E030
:1018A0000E94092ABE016F7077274AE050E080EE5F
:1018B00095E00E94052BDF91CF910895D82FC0E0CD
:1018C000CD1780F42C9A64E670E080E090E00E94EE
:1018D0008B282C9864E670E080E090E00E948B28D2
:1018E000CF5FEECF6CE271E080E090E00E948B2849
:1018F000E6CF0F931F93CF93DF93EC01062F15E0F4
:10190000115051F0CE010E940030081741F0602FB5
:10191000CE010E940830F4CF82E00E945E0CDF917D
:10192000CF911F910F910895A0E0B0E0EAE9FCE0AB
:101930000C94E62D482E562EC0E0D0E0612C712C80
:10194000E12CF12C00E010E041100CC06090D205B9
:1019500086E4689E3001112459E1E52EF12C08EB54
:1019600015E01EC091E049120FC06090D205E6E478
:101970006E9E30011124FBE16F0E711C49E2E42ED2
:10198000F12C04E715E00CC082E0481209C028E100
:10199000622E77247394EE24E394F12C01ED15E08C
:1019A00043018C0E9D1E1092730510927205340136
:1019B000A62CA818B12CC30101966C01AE14BF046B
:1019C000A8F4A00EB11E511006C0C3010E94003041
:1019D000F501808305C0F5016081C3010E94790C87
:1019E000F50180810E9461063601E2CFC3015110EA
:1019F00018C0C3010E940030B82EC6010E940030FA
:101A00002B2D30E0322F2227282B809172059091C8
:101A100073058217930779F4C0E0D0E055245394FE
:101A200093CF3601609173050E94790C6091720525
:101A3000C6010E94790CC05EDE4FC13E92E0D9071C
:101A400008F482CF852DCDB7DEB7E0E10C94022EED
:101A500061E082E00E94940C089560E082E00E94C0
:101A6000940C8091D105853020F01092D1050E9410
:101A7000280D8091D1058093D205089561E080E022
:101A80000E94940C61E081E00E94940C089560E053
:101A900080E00E94940C882351F060E081E00E9475
:101AA000940C882321F080917405883349F00E94BA
:101AB000BF060E947A0681E00E94DF060E943E0D6A
:101AC0000895882319F069EA71E002C06DEA71E0B7
:101AD00080EE95E00E94372A0895FF920F931F939E
:101AE000CF93DF9369EC7BE080EE95E00E94E329E1
:101AF0004091790550917A0560917B0570917C0544
:101B00002AE030E080EE95E00E940C2B63EB7BE056
:101B100080EE95E00E94E32940917D0550917E057D
:101B200060917F057091800520E130E080EE95E0C6
:101B30000E940C2B6DE97BE080EE95E00E94E3298A
:101B40004AE050E06091810580EE95E00E94342BE0
:101B500067E87BE080EE95E00E94E3294AE050E0F0
:101B60006091820580EE95E00E94342B61E77BE076
:101B700080EE95E00E94E329C3E8D5E0F12C8E01C8
:101B800088818823A9F0FF2031F060EB71E080EEBE
:101B900095E00E94062A21964AE050E0F801608113
:101BA00080EE95E00E94FD2AF394F8E1FF12E7CF62
:101BB00080EE95E00E94112A6BE57BE080EE95E0D7
:101BC0000E94E3294AE050E060919B0580EE95E099
:101BD0000E94342B66E47BE080EE95E00E94E329CE
:101BE000E0919C05E770F0E0EE0FFF1FEF57FC4F10
:101BF0006081718180EE95E00E94372A61E37BE08D
:101C000080EE95E00E94E32980919C0588718830E0
:101C100069F028F4811113C068E27BE00CC08031C8
:101C200041F0883161F46CE07BE005C06CE17BE061
:101C300002C066E17BE080EE95E00E94252A68EF15
:101C40007AE080EE95E00E94E3294091750550917D
:101C5000760560917705709178052AE030E080EE96
:101C600095E00E940C2B6FED7AE080EE95E00E94EB
:101C7000E3298091BD0580710E94610D66EC7AE0D8
:101C800080EE95E00E94E3298091BD0580740E945A
:101C9000610D6DEA7AE080EE95E00E94E329809183
:101CA000BD0580720E94610D60E97AE080EE95E0EA
:101CB0000E94E32984E795E00E94F407AB01BC0190
:101CC0002AE030E080EE95E00E94EE2A6BE87AE0B0
:101CD00080EE95E00E94E32984E795E00E94F407F6
:101CE0009B01AC0160E472E48FE090E00E94A32DC0
:101CF000BA01A9012AE030E080EE95E00E94EE2AC8
:101D000068E87AE080EE95E00E94252ACDB7DEB73C
:101D1000E5E00C940D2E8F929F92AF92BF92CF92DE
:101D2000DF92EF92FF92811107C06FE77AE080EEB9
:101D300095E00E94252A2FC090E00E94740724E6B7
:101D400030E040E050E00E94A32DCA01B9012AE032
:101D500030E040E050E00E94A32D49015A016B01A0
:101D60007C012AE030E0B501A40180EE95E00E94FC
:101D7000EE2A6EE280EE95E00E94092A2AE030E029
:101D8000B701A60180EE95E00E94EE2A63E780EE9F
:101D900095E00E94492AFF90EF90DF90CF90BF908E
:101DA000AF909F908F9008951F93CF93DF9365E737
:101DB0007AE080EE95E00E94E32980919D058130D4
:101DC00041F46CE57AE080EE95E00E94252A10E06F
:101DD00050C0823019F465E47AE0F5CF843019F40C
:101DE00061E37AE0F0CF853091F766E27AE0EBCFFD
:101DF000C12FD0E0C930D1050CF441C068E3610FB8
:101E000080EE95E00E94092A6EE17AE080EE95E08E
:101E10000E94E329BE016F5F7F4F4AE050E080EEF1
:101E200095E00E94CD2A63E17AE080EE95E00E9481
:101E3000E329C356DA4FE981E03218F566E07AE02B
:101E400080EE95E00E94E3298981803130F06CE6D4
:101E500073E080EE95E00E94062A69816F7070E061
:101E60006F5F7F4F4AE050E080EE95E00E94D62AF7
:101E70001F5F80914605181708F4BACF0FC061E3C1
:101E8000BECFEF70F0E0EE0FFF1FEF56FC4F60810A
:101E9000718180EE95E00E94372AEACF6BEE79E0FF
:101EA00080EE95E00E94E3298091B5050E948B0E9B
:101EB00060ED79E080EE95E00E94E3298091B6051F
:101EC0000E948B0E65EB79E080EE95E00E94E3299D
:101ED0008091B7050E948B0E6AE979E080EE95E06B
:101EE0000E94E3294091AD055091AE056091AF0588
:101EF0007091B005411551056105710539F12AE070
:101F000030E080EE95E00E940C2B67E679E080EEF1
:101F100095E00E94E3298091B1050E949907AB01E9
:101F2000BC012AE030E080EE95E00E940C2B63E4D7
:101F300079E080EE95E00E94E3294AE050E060916C
:101F4000B20580EE95E00E94342B06C06AE379E08A
:101F500080EE95E00E94252A6DE179E080EE95E023
:101F60000E94E3296091B3057091B4054AE050E006
:101F700080EE95E00E941E2B60E079E080EE95E017
:101F80000E94E3296091AC05603450F470E06F5F0B
:101F90007F4F4AE050E080EE95E00E94D62A06C0CE
:101FA00067EF78E080EE95E00E94252A6AED78E000
:101FB00080EE95E00E94E3298091AB0580FF03C08D
:101FC00062EB71E002C066EB71E080EE95E00E948A
:101FD000372A6DEB78E080EE95E00E94E32980914E
:101FE000AB0582700E94610D6EE978E080EE95E0AD
:101FF0000E94E3298091AB0584700E94610D6FE718
:1020000078E080EE95E00E94E3298091AB0588702E
:102010000E94610DDF91CF911F9108950F931F933F
:10202000CF93DF93209143052F3FA9F56FEF75E024
:1020300080EE95E00E94E32982E893E00E942F0C55
:102040006EED75E080EE95E00E94E32980914405F5
:10205000909145050E942F0C6BEA75E080EE95E0AB
:102060000E94252A68E875E080EE95E00E94252A06
:1020700060E775E080EE95E00E94252A6BE475E04C
:1020800080EE95E00E94252A80EE95E00E94112ABC
:102090000E94D40E68C012160CF065C0332727FDCD
:1020A00030958091460590E0821793070CF45BC051
:1020B00066E375E080EE95E00E94E32960914305B8
:1020C000772767FD70954AE050E080EE95E00E942A
:1020D000D62A6BE075E080EE95E00E94E32910E0DF
:1020E00008E2809147051817D0F5C12FD0E0CC0F3A
:1020F000DD1FC85BDA4F288130E0809143059927C6
:1021000087FD909501972817390739F56AEB71E03B
:1021100080EE95E00E94062A4AE050E0602F80EEB3
:1021200095E00E94FD2A6EEB71E080EE95E00E9442
:10213000062AE981EF70F0E0EE0FFF1FEF56FC4F2B
:102140006081718180EE95E00E94062A62EC71E068
:1021500080EE95E00E94062A0F5F1F5FC2CF80EEDF
:1021600095E00E94112ADF91CF911F910F91089560
:10217000FF920F931F93CF93DF93C3E8D5E0F12C29
:102180008E0188818823D1F164EC71E080EE95E0C6
:102190000E94062A4AE050E06F2D80EE95E00E94F2
:1021A000FD2A61ED71E080EE95E00E94062A2196FD
:1021B000F801208130E0A0E1B7E20E945D2D9B0193
:1021C000AC01A0918205B0E00E946C2DAB01BC0176
:1021D0008091790590917A05A0917B05B0917C055D
:1021E000480F591F6A1F7B1F2AE030E080EE95E000
:1021F0000E940C2BF394F8E1FF12C2CFCDB7DEB7EB
:10220000E5E00C940D2E1092DD0485E6EEEDF4E091
:10221000DF011D928A95E9F70895CF93C82F8F3774
:1022200019F0883009F045C0E091DD04EE23D9F1C2
:10223000E150E093DD04F0E0E252FB4F10826DE0EC
:1022400070E080EE95E00E945906C0E08091DD04C8
:10225000C81760F4EC2FF0E0E252FB4F608170E0B1
:1022600080EE95E00E945906CF5FF0CF60E270E00B
:1022700080EE95E00E9459066DE070E080EE95E0FA
:102280000E945906C0E08091DD04C81778F5EC2F54
:10229000F0E0E252FB4F608170E080EE95E00E943A
:1022A0005906CF5FF0CF67E080EE95E00E94092AE3
:1022B0001DC08B3119F40E9403111AC08D30C1F07A
:1022C0008A30B1F08091DD04843668F76C2F70E0BD
:1022D00080EE95E00E945906E091DD0481E08E0FCA
:1022E0008093DD04F0E0E252FB4FC08380E001C048
:1022F00081E0CF910895CF93C82F0E946828609302
:10230000C6047093C7048093C8049093C904C09313
:10231000DB04CC2329F040E051EE60E070E004C023
:1023200040E855E260E070E080EE95E00E94932C7A
:10233000CF9108959091CA04492F4F7050E0BA018F
:102340006F5F7F4F292F30E0E4E035952795EA95C0
:10235000E1F76217730759F0FA01E553FB4F8083E9
:1023600081E0890F8F70907F892B8093CA04089534
:102370006EE770E080EE95E00E9459060895A3E1B3
:10238000B1E0E5ECF1E10C94E72DE3E8F5E0712C28
:102390008191882321F0739428E17212F9CF65EDC1
:1023A00071E080EE95E00E94372A4AE050E0672D08
:1023B00080EE95E00E94342B80E00E947D0A0E940E
:1023C000580B8E010E5F1F4FC12CD12C7601C39488
:1023D00066246A945C2C0E945C284B015C0120916D
:1023E000820530E0A0E1B7E20E945D2D9B01AC01C7
:1023F000C701B6010E947F2D2091790530917A05A1
:1024000040917B0550917C05620F731F841F951FBF
:102410002091B9053091BA054091BB055091BC059A
:10242000261737074807590718F4F801608225C0B6
:102430008C2D0E94B10961E070E080E090E00E9484
:102440008B28F80110820E945C28681979098A0992
:102450009B09643F71408105910540F40E94C709C2
:10246000F8019081981778F78083EDCF50FE03C074
:102470002B982C9A02C02B9A2C982FEFC21AD20AB2
:10248000E20AF20A0F5F1F4F8FEFC816D104E10472
:10249000F10409F09FCFCE019395FC01D82E7FEF78
:1024A00068EC2E2F281B271510F051E056C0DE01D6
:1024B000129651E02FEF41E03D91321710F0322F8C
:1024C00001C0452F5F5F5F3F11F0232FF5CF419390
:1024D000242F30E0A1E0B0E0AC0FBD1FA20FB31F6E
:1024E0005C93413079F0DE01A20FB31F5C93423060
:1024F00049F0AFEFBFEFAC0FBD1FA20FB31F6C933E
:102500004E3F78F6A2E0B0E0AC0FBD1FA20FB31FA4
:102510007C934D3F30F6A3E0B0E0AC0FBD1FA20F9F
:10252000B31F6C93BECF452F242F30E0FC01E20F88
:10253000F31F6081AFEFB0E0AC0FBD1FA20FB31F60
:102540002C91621748F44150DC01A40FB11D2C916D
:1025500020836C934111E8CF5F5F571520F3372D2F
:10256000369520E0231770F4DC01A20FB11D4C91C9
:10257000522F530FFC01E50FF11D50815C934083F6
:102580002E5FF0CFF3E8EF2EF5E0FF2E8C01802FC9
:102590008D19871598F4F801C1908F014AE050E039
:1025A0006C2D80EE95E00E94FD2A6CE280EE95E0B5
:1025B0000E94092AF701C1927F01E9CF80EE95E0E0
:1025C0000E94112A81E0CD5EDE4FEFE00C94032ED5
:1025D0001F920F920FB60F9211240F931F932F93F8
:1025E0003F934F935F936F937F938F939F93AF939B
:1025F000BF93EF93FF934091BD055091BE0560914D
:10260000BF057091C00586B18A019B010074112736
:102610002227332785FB882780F990E0A0E0B0E0EF
:10262000081719072A073B0709F468C0809184003E
:102630009091850010928500109284002091A7044B
:1026400021115CC045FD02C096958795853C29E027
:102650009207C0F180910A0190E0A0E0B0E00CE1A7
:1026600076956795579547950A95D1F74115510588
:102670006105710521F441E050E060E070E0481729
:1026800059076A077B07D8F480910A018F3FB9F098
:1026900040E080910A01481780F4842F90E0880F71
:1026A000991FFC01E957FB4F20813181FC01E55F57
:1026B000FE4F318320834F5FECCF1092A80410921D
:1026C0000A011CC08D3B22E09207A8F020910A016C
:1026D000203188F410910A0121E0210F20930A0192
:1026E0000E94DE08E12FF0E0EE0FFF1FE957FB4FDD
:1026F0009183808303C08FEF80930A01FF91EF9154
:10270000BF91AF919F918F917F916F915F914F9109
:102710003F912F911F910F910F900FBE0F901F901F
:10272000189583E0809380008AE1809381008FEF89
:102730009FEF909389008093880010926F0080E251
:1027400080936C00E8E6F0E08081826080830895E9
:102750000E942D0D8091D205843011F41092D20583
:1027600008956F3018F086958058089589E0689F25
:10277000802D11240895A0E0B0E0E1ECF3E10C9489
:10278000EE2DC82F0E94682800913804109139045A
:1027900020913A0430913B046B017C01C01AD10AAC
:1027A000E20AF30A9701860149E8C41643E1D40618
:1027B000E104F10410F010923C046093380470932B
:1027C000390480933A0490933B042091A7048FEF3F
:1027D000820F8230D8F5E0913C04EE2309F44EC11B
:1027E000E13011F482E0B8C1E03108F034C181E099
:1027F0008E0F80933C04F0E0E957FB4FC08380319B
:1028000009F0ACC1E9E8F4E0213029F4A181A695F2
:10281000A695808108C080819181A92FA695A69553
:10282000A69596958795A03148F4B0E090E0AA0F60
:10283000BB1FA55FBE4F11969C938E931092A80468
:10284000329684E0E739F807F9F688C1233009F0B9
:1028500005C1E0913C04E11104C0CF3009F07EC114
:102860000DC1E83148F481E08E0F80933C04F0E024
:10287000EA57FB4FC08372C1E83109F0ECC0C111C7
:10288000EAC040E050E0ABE0CA01B3E0880F991F16
:10289000BA95E1F7A49F9001A59F300D1124F9018D
:1028A000E957FB4F6081E1817E2F777075956795C1
:1028B000FC01EE0FFF1FE55FFE4F71836083F9019E
:1028C000E857FB4FB081B695B695B695E181FE2FDE
:1028D000F295FF0FF07E6F2F6B2BE695E695E69550
:1028E0007E2F777075956795FC01EE0FFF1FE35FF4
:1028F000FE4F71836083F901E757FB4FB081B295BA
:10290000B695B695B370C181DC2FDD0FDD0F6D2F4D
:102910006B2BC295C695C695C370E281E170EE0F30
:10292000EE0F7E2F7C2B75956795FC01EE0FFF1F38
:10293000E15FFE4F71836083F901E557FB4FB08182
:10294000B695E181FE2FF795FF27F7956F2F6B2B3B
:10295000E6957E2F777075956795FC01EE0FFF1F4A
:10296000EF5EFE4F71836083F901E457FB4FB08146
:10297000B295BF70E181FE2FF295F07F6F2F6B2B28
:10298000E295EF707E2F777075956795FC01EE0FDD
:10299000FF1FED5EFE4F71836083F901E357FB4F2C
:1029A000B081BB1FBB27BB1FC181DC2FDD0F6D2F8B
:1029B0006B2BCC1FCC27CC1FE281E370EE0F7E2F58
:1029C0007C2B75956795FC01EE0FFF1FEB5EFE4FAC
:1029D00071836083F901E157FB4FB081B695B695DD
:1029E000E181FE2FF295FF0FFF0FF07C6F2F6B2B15
:1029F000E695E6957E2F777075956795FC01EE0F4D
:102A0000FF1FE95EFE4F71836083F901E057FB4FC2
:102A100020812295269527703181E32FEE0FEE0F4E
:102A2000EE0F6E2F622B732F7295769577707595DA
:102A30006795FC01EE0FFF1FE75EFE4F7183608319
:102A40004F5F5F4F4230510509F01ECF80919D04CA
:102A500083FF1092A80410923C0480C0243009F037
:102A60007DC060913C0461110BC0C83AB1F4109272
:102A700073051092720588EA0E94610681E06CC0BD
:102A8000613019F4C093370404C0623031F4C0934C
:102A900036048C2F0E9461065AC0E09136042E2F16
:102AA00030E0220F331F462F50E0C90102968417F1
:102AB00095073CF0633268F7FA01EC57FB4FC0838F
:102AC000E8CF2D5F3F4F8C2F90E0609172057091A1
:102AD00073054217530749F4982F882786279727AD
:102AE000909373058093720532C06817790769F572
:102AF00080913704813049F5E13118F080E180930D
:102B00003604F0903604C8E8D4E000E010E00F1579
:102B1000D0F4FE013197808190E0982F882728819A
:102B2000822B43E0969587954A95E1F70E94DE084F
:102B3000F801EE0FFF1FE55FFE4F918380830F5F6B
:102B40001F4F2296E4CF1092A80410923C0480916B
:102B50003C04882319F08F5F80933C04CDB7DEB727
:102B6000E8E00C940A2EE82FF0E0E854FA4FE185F3
:102B7000E03150F4F894F0E0EE0FFF1FE55FFE4FF8
:102B8000808191817894089580E092E00895A2E296
:102B9000B0E0EDECF5E10C94E42D9E012F5F3F4F8A
:102BA00080E1D9011D928A95E9F763E072E080EE39
:102BB00095E029A33AA30E94372A0E947B0B1D8A25
:102BC0001E8A1F8A188E312C212C00E0812C912C1A
:102BD000540170EC472E7DE9572E78E5672E75E39A
:102BE000772EE0E5CE2EE3ECDE2EE12CF12C84EF07
:102BF00091E0A0E0B0E08D8F9E8FAF8FB8A380EC06
:102C000097EFAAEBB7E3898F9A8FAB8FBC8F80ECDD
:102C10009DE9A8E5B5E3898B9A8BAB8BBC8B80EEE5
:102C200095E00E944B2B892B09F4E1C080EE95E0E2
:102C30000E94782B9C0133272C32310509F442C0C5
:102C4000ACF42332310509F0ABC019821A821B8221
:102C50001C821D821E821F82188619861A861B8678
:102C60001C861D861E861F86188A60C02434310586
:102C700029F02335310509F4B2C092C064E480EE36
:102C800095E00E94092A2AE030E040EC5DE968E521
:102C900075E380EE95E00E94972A6CE280EE95E065
:102CA0000E94092A2AE030E040EC57EF6AEB77E314
:102CB00080EE95E00E94972A6CE280EE95E00E94FB
:102CC000492AADCF0F5F043009F0A9CF29813A819D
:102CD0004B815C81A8EEB3E00E946C2D698B7A8BEE
:102CE0008B8B9C8B2D813E814F8158850E946C2D52
:102CF000698F7A8F8B8F9C8F29853A854B855C8570
:102D00002D8F3E8F4F8F58A32D853E854F85588937
:102D10000E946C2D6B017C0160323EE473078105DB
:102D2000910530F462E38CE10E949E0900E077CFC8
:102D3000603345E774078105910510F462E2F3CF33
:102D400060345CE975078105910510F466E2EBCF0C
:102D500080E5C81683ECD806E104F10410F462E1C2
:102D6000E2CF90E6C9169AEED906E104F10410F418
:102D700065E1D9CFA0E7CA16A1E1DA06A1E0EA062B
:102D8000F10410F461E0CFCFB0EACB16B6E8DB0671
:102D9000B1E0EB06F10410F463E0C5CF65E0C3CF0A
:102DA00010ED180F1A3008F03ACFE1E0F0E0EC0F28
:102DB000FD1F24E0029FE00DF11D112420813181CF
:102DC00042815381AAE0B0E00E946C2D610F711D19
:102DD000811D911D608371838283938320CF4988F5
:102DE0005A886B887C88812C912C540118CF8114CF
:102DF0009104A104B10489F4C301B2010E940D0A37
:102E000061E070E080E090E00E948B281D8A1E8ABD
:102E10001F8A188E312C22242A948D8D9E8DAF8D81
:102E2000B8A188169906AA06BB06D0F40E94C70965
:102E30002D893E894F89588D280F311D411D511D07
:102E40002D8B3E8B4F8B588F381608F4382E8215F9
:102E500008F4282E3FEF831A930AA30AB30A56C038
:102E6000C301B20128EE33E040E050E00E94A32D00
:102E7000BA01A9012AE030E080EE95E00E94EE2A36
:102E80006CE280EE95E00E94092A4AE050E0632D52
:102E900080EE95E00E94FD2A6CE280EE95E00E94B3
:102EA000092A6D897E898F89988DA50194010E94D8
:102EB000A32DBA01A9012AE030E080EE95E00E943E
:102EC000EE2A6CE280EE95E00E94092A4AE050E08A
:102ED000622D80EE95E00E94FD2A6CE280EE95E086
:102EE0000E94492A4C0C5D1C6E1C7F1C898D9A8D9A
:102EF000AB8DBC8D84159505A605B70520F44988D2
:102F00005A886B887C88812C912C540129893A89B4
:102F10004B895C89283E33404105510509F07FCE3D
:102F2000A296E2E10C94002EACE1B0E0EAE9F7E110
:102F30000C94EE2D0E9468286B017C0181E00E94B8
:102F40007D0A14E703E0198361E0CE0101960E9437
:102F5000DA0B009371050E94580B6AEF70E080E075
:102F600090E00E948B2880917105833089F480EE77
:102F700095E00E944B2B892B59F40E9468286C190C
:102F80007D098E099F096038734C894C9140D8F2B5
:102F900080917105833009F44FC08FE70E94760954
:102FA0000E9489098983843511F083E05CC00E9406
:102FB000890910924405809345050E948909209152
:102FC000440530914505280F311D30934505209368
:102FD00044050E948909809346050E9489098093CF
:102FE0004705813110F7F12C0F2D10E08091470536
:102FF00090E0880F991F0817190740F40E9489096B
:10300000F801E85BFA4F8083F394EECF80E7898381
:1030100061E0CE0101960E94DA0B83E08093710596
:103020000E94580B62E370E080E090E00E948B28E1
:1030300080917105833011F482E015C08FE70E9402
:1030400076090E9489098983803509F0AECF0DE9A0
:1030500015E00E948909F80181938F01F5E0083B92
:103060001F07B9F781E06C96E8E00C940A2E809176
:103070004305992787FD9095A92FB92FFC0131961B
:10308000EB30F10508F066C0EC5CFF4F0C941B2E92
:1030900062E778E080EE95E00E94252A82E893E0DE
:1030A0000E942F0C6AE578E080EE95E00E94252AC8
:1030B00065E378E080EE95E00E94252A6BE078E0F9
:1030C00080EE95E00E94252A6AEE77E080EE95E09A
:1030D0000E94252A6DEB77E080EE95E00E94252A7C
:1030E00067E977E080EE95E00E94252A63E777E0C4
:1030F00080EE95E00E94252A6CE477E080EE95E072
:103100000E94252A80EE95E00E94112A0E946D0DF2
:1031100021C06FE277E01AC06AE077E017C065EF80
:1031200076E014C066ED76E011C062E976E00EC08C
:103130006DE776E00BC068E676E080EE95E00E94F1
:10314000252A62E276E002C06CE076E080EE95E04F
:103150000E94252A6AE070E080E090E00E948B28BF
:1031600080EE95E00E944B2B892B29F080EE95E0B4
:103170000E94782BF5CF0895ACE1B0E0E2ECF8E1E5
:103180000C94EE2D909143059F3F09F023C1482FE9
:1031900050E0FA013A97EF36F10508F00FC1E15C13
:1031A000FF4F0C941B2E60E172E0A0C06CE172E056
:1031B00080EE95E00E94372A85E789838BE1EDE96F
:1031C000F5E0DE01129601900D928A95E1F76CE12F
:1031D000CE0101960E94DA0B0E94580B83E0809387
:1031E000710568EC70E080E090E00E948B2880918F
:1031F0007105843009F0E2C08FE70E9476090E94D1
:1032000089098983853509F0D9C06DEE74E080EEB7
:1032100095E00E94252A6FEC74E080EE95E00E9414
:10322000252A61EB74E096C064E372E080EE95E0DD
:103230000E94372A89E6898361E0CE0101960E94C7
:10324000DA0B0E94580B83E08093710568EC70E004
:1032500080E090E00E948B2880917105843009F015
:10326000ADC08FE70E9476090E94890989838E018B
:103270000E5F1F4F7E014DE1E40EF11C0E94890993
:10328000F80181938F01EE15FF05C1F78BE1FE0177
:103290003296ADE9B5E001900D928A95E1F789810A
:1032A000893409F08BC063E974E080EE95E00E94F8
:1032B000252A65E774E080EE95E00E94252A67E5FF
:1032C00074E048C06EE472E080EE95E00E94372A18
:1032D0008EEF8093430572C0805287508053909147
:1032E0004605981708F066C06DE572E080EE95E03F
:1032F0000E94372A63C084E18093430560E274E052
:1033000029C085E18093430569EE73E023C086E11F
:103310008093430562EB73E01DC087E18093430512
:1033200068E673E017C088E18093430567E573E0C2
:1033300011C089E18093430563E473E00BC08AE127
:10334000809343056EE273E005C08BE180934305F3
:1033500066E073E080EE95E00E94252A2FC06CEEB7
:1033600072E080EE95E00E94252A8091AB0591E005
:103370001DC066ED72E080EE95E00E94252A8091E6
:10338000AB0592E013C061EC72E080EE95E00E9424
:10339000252A8091AB0594E009C066EA72E080EED0
:1033A00095E00E94252A8091AB0598E089278093BB
:1033B000AB058FEF809343050E940E1080EE95E0E1
:1033C0000E944B2B892B09F45BC180EE95E00E9493
:1033D000782BF4CF0E940D11882309F451C18091FC
:1033E000DD04811104C08FEF8093430541C140E0AB
:1033F00050E060E070E08EED94E00E94922E4091EB
:103400004305042F112707FD1095212F312FF801B7
:103410003197EB31F10508F01BC1E255FF4F0C94D9
:103420001B2E552747FD50952091460530E0241767
:1034300035070CF40DC18B019C01015011092109C4
:103440003109003211052105310558F0C0904705BA
:10345000E9E4F5E0F12CD12CA8E2EA2E4150510923
:103460000FC0FA01E356FA4F61506083D9C0DF0103
:1034700011972C9130E02417350729F0F3943296F8
:10348000FC10F5CFCBC00E2D10E020E030E0061789
:1034900017072807390741F42081DA01A356BA4FEC
:1034A00011962C93DD24D394E394E8CF6F3F7105FC
:1034B0008105910511F008F0CBC06093B505B0C04F
:1034C0006F3F71058105910511F008F0C1C060934F
:1034D000B605A6C06F3F71058105910511F008F092
:1034E000B7C06093B7059CC02091DE0420622037EE
:1034F000E9F440E050E060E070E08FED94E00E947D
:10350000922E9B01AC01DC01CB010197A109B1090D
:103510000897A105B10508F0AEC0A4EDB0E30E9484
:103520006C2D6A5E7C4A8A46954E24C02636E9F4A4
:1035300040E050E060E070E08FED94E00E94922E59
:103540009B01AC01DC01CB010197A109B1090797EF
:10355000A105B10508F08FC0A8EAB1E60E946C2D64
:10356000645E7C438E46944E05C0611571058105ED
:10357000910579F08B019C01005C1D49284535437C
:103580000130FAE51F07F2E62F07F2E03F0708F0E7
:103590005FC06093AD057093AE058093AF059093C7
:1035A000B0053EC06F3F71058105910511F008F02F
:1035B0004FC06093B10534C08B019C0101501109CB
:1035C000210931090F3F11052105310508F040C0DF
:1035D0006093B20525C08B019C01045C1940210950
:1035E00031090D344DE114072105310528F470939C
:1035F000B4056093B30514C061157105810591058B
:1036000021F48FEF8093AC050BC061347105810507
:103610009105F0F461506093AC0502C0DD20C1F06B
:103620008091DC0481111AC080917D0590917E0506
:10363000A0917F05B09180050196A11DB11D8093D9
:103640007D0590937E05A0937F05B093800506C00D
:103650006FE672E080EE95E00E94372A0E94031127
:103660008FEF809343056AE080EE95E00E94492A3F
:103670000E940E1005C061E070E080E090E07ACF1B
:103680006C96E8E00C940A2E6AE572E080EE95E014
:103690000E94252A62E472E080EE95E00E94252ACD
:1036A00080EE95E00E944B2B892B31F080EE95E067
:1036B0000E94782B0E94BC180E949417823029F037
:1036C000833051F46DE072E002C064E272E080EE9B
:1036D00095E00E94252A08958FEF8093430510926C
:1036E000DC040E940E10809143058E3F69F080EE4D
:1036F00095E00E944B2B892BB1F380EE95E00E9460
:10370000782B0E94BC18EFCF08950F931F93109150
:1037100043051F3F09F0D2C0893409F457C000F5B2
:10372000883309F469C058F4803309F477C008F08D
:1037300061C08B3109F440C08132B1F1B9C081342C
:1037400009F487C030F4893309F466C0803461F12C
:10375000AFC0823409F48EC0863409F448C0A8C0D2
:10376000823609F487C078F4883531F128F482353F
:10377000C1F18335E1F09CC08A3509F494C08136EB
:1037800009F467C095C0823761F128F4863679F173
:103790008936E1F08DC0883779F08A3709F483C023
:1037A000833709F085C003C060E172E015C00E9454
:1037B0003E0D6DE872E004C00E94470D67EA72E0BA
:1037C00080EE95E00E94372A8EEF70C00E947A0644
:1037D0000E94BF0666EC72E080EE95E00E94372AF8
:1037E00067C081E00E94DF066FED72E0F5CF0E94B6
:1037F000B8105EC080535AC06AEF71E080EE95E069
:103800000E94252A90919C0588E0890F8871977EF7
:10381000892B80939C051AC089E048C067EE71E04F
:1038200080EE95E00E94252A8091BD059091BE050D
:10383000A091BF05B091C00520E182278093BD050E
:103840009093BE05A093BF05B093C00510934305A8
:103850002FC061ED71E080EE95E00E94252A8091F5
:10386000BD059091BE05A091BF05B091C00540E493
:10387000842710C060EC71E080EE95E00E94252A5C
:103880008091BD059091BE05A091BF05B091C00586
:1038900020E282278093BD059093BE05A093BF05CB
:1038A000B093C00502C00E94441B8FEF8093430574
:1038B000809143058E3F09F0D4C0DDC00E940D11F8
:1038C000882309F4D8C08091DD04811104C08FEFF2
:1038D00080934305C6C040E050E060E070E08EEDAC
:1038E00094E00E94922E00914305112707FD109548
:1038F000212F312FF8013197E930F10508F0B4C0DC
:10390000E753FF4F0C941B2E8B019C01015C1D495A
:10391000284535430F3F19452246324008F0A4C0E0
:103920006093790570937A0580937B0590937C056D
:1039300077C060937D0570937E0580937F0590939B
:10394000800581E08093DC046BC0683071058105DF
:10395000910508F089C06093810562C08B019C01CC
:1039600001501109210931090A30110521053105DC
:1039700008F07AC06093820553C060EB71E08EED71
:1039800094E00E94CC2F10E0009799F00E94A62F9F
:10399000009779F0183130F4E12FF0E0EC58FA4F4D
:1039A00087871F5F60EB71E080E090E00E94CC2F82
:1039B000EBCF1831A8F5E12FF0E0EC58FA4F17865D
:1039C0001F5FF7CF653071058105910508F04CC088
:1039D00060939B0525C08B019C01015011092109B1
:1039E00031090630110521053105F0F520919C05BE
:1039F000287F262B20939C0513C08B019C0101502E
:103A00001109210931090115124C2140310560F5D8
:103A1000609375057093760580937705909378058C
:103A20008091DC04811113C080917D0590917E0509
:103A3000A0917F05B09180050196A11DB11D8093D5
:103A40007D0590937E05A0937F05B09380050E942D
:103A500003118FEF809343056AE080EE95E00E94AA
:103A6000492A0E94371807C06FE672E080EE95E0A1
:103A70000E94372AECCF1F910F9108958FEF80930A
:103A800043051092DC040E943718809143058E3F55
:103A900069F080EE95E00E944B2B892BB1F380EE0C
:103AA00095E00E94782B0E94851BEFCF6AE070E0C2
:103AB00080E090E00E948B2880EE95E00E944B2BE6
:103AC000892B29F080EE95E00E94782BF5CF0895A0
:103AD000CF93C82F682F80EE95E00E94A52B909180
:103AE00068059C2790936805CF910895A1E0B0E008
:103AF000ECE7FDE10C94F42D99830E94681D9981F7
:103B0000892F0E94681D2196E2E00C94102E1F93CD
:103B1000CF93DF93182FEB011092680565EB70E0EF
:103B200080EE95E00E94590662E670E080EE95E036
:103B30000E945906812F0E94681DCE010E94761DA9
:103B4000DF91CF911F9108956091680580EE95E017
:103B50000E94A52B0895A1E2B0E0E1EBFDE10C94F9
:103B6000F02D7B018A018C3009F453C108F040C06C
:103B7000863009F4BCC018F5833009F491C070F4A4
:103B8000813009F472C0823009F048C26BE170E004
:103B900082E00E94871D0DE915E078C0843009F4A9
:103BA00087C0853009F03AC26091470570E0660F22
:103BB000771F85E00E94871D08E415E086C08930E4
:103BC00009F4A7C070F4873009F49BC0883009F06D
:103BD00025C261E070E088E00E94871D8091D205D7
:103BE00023C28A3009F4CAC08B3009F4F2C016C26D
:103BF0008A3609F475C1D8F4873609F43AC138F425
:103C0000853609F40EC1863609F41FC107C288360D
:103C100009F437C1893609F001C261E070E089E634
:103C20000E94871D0E947A060E94BF06F5C18D364C
:103C300009F4D4C138F48B3609F491C18C3609F4F7
:103C40009AC1ECC18E3609F4DCC1873C09F0E6C1AB
:103C500061E070E087EC0E94871D81E00E94681D92
:103C60000E94A41D10926905E3C169E270E081E041
:103C70000E94871D04E715E0F80181918F010E94E1
:103C8000681DF5E00D391F07B9F7D0C1F801819122
:103C90008F010E94681DF5E0083B1F07B9F7C6C1F8
:103CA00061E070E083E00E94871D0E949417BCC110
:103CB00061E070E084E00E94871D81E00E94681D41
:103CC0000E94A41D0E94C715B3C18091470590E0D2
:103CD000880F991F9801285435402817390708F094
:103CE000A5C1F80181918F010E94681DEECF62E0AD
:103CF00070E086E00E94871D82E893E00E94761DB6
:103D000095C161E070E087E00E94871D80914605C3
:103D10008BC186E6898361E0CE0101960E94DA0BB1
:103D20000E94580B83E08093710568EC70E080E09E
:103D300090E00E948B28809171058430D9F48FE740
:103D40000E9476090E9489098983863469F460E2B9
:103D500070E089E00E94871D10E20E9489090E949C
:103D6000681D1150D1F762C161E070E089E00E94E6
:103D7000871D52C161E070E089E053C169E170E0E4
:103D80008AE00E94871D82E08093B805209170052B
:103D90008091BD059091BE05A091BF05B091C00571
:103DA000222311F0806801C08F778093BD05909326
:103DB000BE05A093BF05B093C00508EB15E0F80160
:103DC00081918F010E94681DF5E0013D1F07B9F741
:103DD0002DC161E270E08BE00E94871D8091A804F4
:103DE0008F3F39F08091A80491E0980F9093A80438
:103DF00002C08091A8040E94681D10E0812F0E94DB
:103E0000B3150E9409090E94761D1F5F1031B1F79A
:103E10000DC161E070E08CE00E94871D8091D105AA
:103E200003C161E070E085E60E94871D89E2E81623
:103E3000F10409F0F8C0D801E4E7F5E08D91819331
:103E400085E0ED39F807D1F7E7C061E070E086E67C
:103E50000E94871DEBE1EE16F10409F0E4C0D801E1
:103E6000EDE9F5E08D91819385E0E83BF807D1F726
:103E7000D3C061E070E087E60E94871D0E943E0D7E
:103E8000CBC061E070E088E60E94871D85E78983EA
:103E90008BE1EDE9F5E0DE01129601900D928A9535
:103EA000E1F76CE1CE0101960E94DA0B0E94580BFB
:103EB00083E08093710560E273E080E090E00E940F
:103EC0008B2880917105843009F0ADC08FE70E9486
:103ED00076090E9489098983853509F0A4C09CC0B0
:103EE00061E070E08AE60E94871D89E6898361E0CF
:103EF000CE0101960E94DA0B0E94580B83E080935A
:103F0000710560E273E080E090E00E948B28809170
:103F10007105843009F087C08FE70E9476090E94FE
:103F2000890989838E010E5F1F4F7E01EDE1EE0E40
:103F3000F11C0E948909F80181938F01EE15FF059C
:103F4000C1F78BE1FE013296ADE9B5E001900D922B
:103F50008A95E1F78981893409F065C05DC061E027
:103F600070E08BE60E94871DF80180818093D20566
:103F70000E94470D51C061E070E08CE60E94871DF1
:103F8000F0E2EF16F10461F487E6898380E2F8013C
:103F9000DE01129601900D928A95E1F761E203C06D
:103FA00087E4898361E0CE0101960E94DA0B0E94CA
:103FB000580B83E0809371056CE474E080E090E03E
:103FC0000E948B2880917105843069F58FE70E94EB
:103FD00076090E948909873431F51EC061E070E0DE
:103FE0008DE60E94871D89E1E816F104E1F4D8010D
:103FF000E8EBF5E08D91819385E0E13DF807D1F79D
:104000000BC061E070E08EE60E94871DF8018081A0
:104010008093D1050E94280D81E006C061E070E028
:104020008AEC0E94871D80E00E94681D0E94A41DEA
:10403000A196E6E00C940C2EA0E0B0E0E2E2F0E203
:104040000C94EE2DCAECD3E014E606E035E0F32E36
:1040500044E0E42E53E0D52E62E0C62E80EE95E0DB
:104060000E944B2B892B09F49BC080EE95E00E94A7
:10407000782B282F809335044091340450E047304A
:10408000510560F7FA01EE52FF4F0C941B2E853B51
:1040900029F781E080933404E1CF823609F07DC0B6
:1040A000C0923404DBCF8093330480933204D092E7
:1040B0003404D4CF9C01332730933104209330044F
:1040C00090913204982790933204E0923404C6CF42
:1040D000382F22274091300450913104242B352B66
:1040E00030933104209330049091320498279093B8
:1040F0003204F09234042536310508F4AFCF61E084
:1041000070E08CEC0E94871D81E00E94681D0E9477
:10411000A41D43C020912E0430912F04F901E653D1
:10412000FC4F808390913204982790933204C90108
:10413000019690932F0480932E04209130043091A7
:1041400031048217930708F489CF0093340486CF93
:104150008091320482130BC060912E0470912F0461
:104160004AEC53E0809133040E94AB1D0DC062E025
:1041700070E08BEC0E94871D809133040E94681DC3
:10418000809168050E94681DFE01812F11928A9519
:10419000E9F710922F0410922E04109234045ECF8F
:1041A000CDB7DEB7E8E00C940A2E81E08093690574
:1041B00080916905882349F080EE95E00E944B2BA1
:1041C000892BB1F30E941C20F3CF0895AAE2B0E03E
:1041D000ECEEF0E20C94EC2D0E945C286B017C016B
:1041E00081E00E947D0A80EE95E00E944B2B892B96
:1041F00029F080EE95E00E94782BF5CF2C9811E005
:1042000072E6B72EE9E2AE2E03E00E945C286C193C
:104210007D098E099F09693C710581059105D0F1E1
:104220001123C1F10E945C286B017C012B9A80ED67
:1042300097E00E94A807B982E4E7F5E0DE01129654
:104240008A2D01900D928A95E1F76AE2CE010196DE
:104250000E94DA0B2B9880E090E00E94A807009360
:1042600071050E94580B62E370E080E090E00E94CC
:104270008B2880917105843061F4009371058FE77C
:104280000E9476090E94890911E0823419F410E035
:1042900001C011E08AE00E948129892B81F411E09C
:1042A0000EC02C9A2B9A80EE95E00E94782B8D30D0
:1042B0009105A9F05CF40A9791F02C982B9880EE68
:1042C00095E00E944B2B892B61F79FCF833291059C
:1042D00079F08234910589F70E94D520EECF62EB08
:1042E00071E080EE95E00E94252A0E943E1DE5CFF8
:1042F0000E94C715E2CF8F929F92AF92BF92CF924A
:10430000DF92EF92FF921F93CF93DF938AE00E9498
:104310008129892B09F089C068EC70E080E090E089
:104320000E948B2880E090E00E94A8070E945C28F1
:104330004B015C016B017C0180ECC80E82E1D81E50
:10434000E11CF11C0E945C286C157D058E059F0503
:1043500030F48AE00E948129892BA1F364C08AE0AD
:104360000E948129892B09F05EC080ED97E00E94B0
:10437000A8070E945C286B017C01D0E0C1E088E4C2
:10438000880E86E2981EA11CB11C11E08AE00E94F2
:104390008129892B21F58C149D04AE04BF0430F4CF
:1043A00080ED97E00E94A807D1E0F0CF0E945C2842
:1043B0006C197D098E099F09693C7105810591057C
:1043C00028F30E945C286B017C01C12719F080ED65
:1043D00097E002C080E090E00E94A807D7CF80E07D
:1043E00090E00E94A807DD23B9F08091D10590E00C
:1043F000019665E070E00E948F2D8093D1050E94A8
:10440000280D0E94A8130E94470D64EF71E080E020
:1044100090E00E948B2809C080E00E94DF060E9485
:10442000BF110E943E0D0E94E620DF91CF911F91A7
:10443000FF90EF90DF90CF90BF90AF909F908F90C4
:104440000895CF92DF92EF92FF9280E00E94DA0708
:104450000E94B10761E08CE00E94152961E08BE0C9
:104460000E94152960E08AE00E94152960E083E13E
:104470000E94152961E083E10E944E2961E082E1FA
:104480000E94152960E082E10E944E290E949F0748
:1044900040E052EC61E070E080EE95E00E94932CE9
:1044A0000E94A8130E94470D0E9491138FEF8093E2
:1044B000A8040E94C60778940E945C286B017C01C6
:1044C0008091A8048F3F59F40E945C286C197D09E3
:1044D0008E099F09603D77408105910588F380ED45
:1044E00097E00E94A80761E08AE00E944E292C9A7A
:1044F00080EE95E00E944B2B892B29F080EE95E011
:104500000E94782BF5CF6CEF72E080EE95E00E9470
:10451000062A82E893E00E942F0C63E173E080EEAC
:1045200095E00E94062A4AE050E060E070E080EEEC
:1045300095E00E94D62A62E370E080E090E00E945D
:104540008B2880EE95E00E944B2B04970CF180EEB7
:1045500095E00E94782B82349105D1F480EE95E0AD
:104560000E94782B8E34910599F480EE95E00E949C
:10457000782B8434910561F480EE95E00E94782BCD
:10458000819731F480E090E00E94A8070E94E62025
:104590004091750550917605609177057091780589
:1045A000DB01CA010197A109B1090497A105B10571
:1045B00068F44093A704433029F440EA56E861E0E8
:1045C00070E004C040E052EC61E070E080EE95E005
:1045D0000E94932C0E947B212C9880E090E00E9406
:1045E000A8070E9491131092C3048091BD0583FF18
:1045F00011C080918905882351F08091900588230E
:1046000031F080919705882311F087E001C085E0A3
:104610008093C30480E00E947D0A8091C4040E94BC
:10462000B1090E94580B10923F0410923E04109260
:104630003D04F12C8091D2058F15B0F062E370E05B
:1046400080E090E00E948B2880ED97E00E94A80710
:1046500062E370E080E090E00E948B2880E090E0D0
:104660000E94A807F394E6CF80919C0584FF08C0C0
:10467000982F987181E0983109F080E00E947B11B9
:104680008FE00E94DA07FF90EF90DF90CF900895BF
:10469000EF92FF920F931F93CF93DF938C016EE7FE
:1046A00070E080EE95E00E945906E801F12CF0E2FE
:1046B000EF2E8E0188818D57823048F46DE770E0CF
:1046C00080EE95E00E94590688818E258883219688
:1046D000F801608180EE95E00E94A52BF394F9E04B
:1046E000FF12E7CF6EE770E080EE95E00E9459067A
:1046F000CDB7DEB7E6E00C940C2EA9E0B0E0E3E81D
:10470000F3E20C94F42D9091C50491110EC09EEF2C
:1047100099838A836B8350E0559547954C832D830D
:10472000198618861F821E822EC04091CA04842FCB
:1047300090E0B4E095958795BA95E1F7242F2F7016
:1047400030E08217930719F18DEF89831B82FE01F8
:10475000349650E0842F90E0A4E095958795AA9533
:10476000E1F7242F2F7030E08217930749F0DC0126
:10477000A553BB4F8C918193405F5F5F563051F7DB
:104780004093CA045A83CE0101960E944823809127
:10479000C50490E0019666E070E00E948F2D809342
:1047A000C5042996E2E00C94102EA0E0B0E0EBEDF9
:1047B000F3E20C94ED2D6C016EE770E080EE95E075
:1047C0000E9459068601E12CF12CC0E0D0E030E2D5
:1047D000B32EF801608183E8860F823078F46DE7AC
:1047E00070E080EE95E00E945906F80160816B252B
:1047F00070E080EE95E00E94590604C080EE95E0DE
:104800000E94A52BE114F10459F0F80180819E016A
:10481000280F311DC901C92FDD27C80FD91FDD277A
:104820003FEFE31AF30A89E0E816F10459F028E0B3
:10483000E216F10421F48C2F8095F60180870F5F3A
:104840001F4FC7CFCDB7DEB7E9E00C94092EA9E022
:10485000B0E0EDE2F4E20C94F42DE82F362F8091D5
:10486000C50490E0019664E270E00E948F2D809371
:10487000C50458E9598350E15A83813089F048F0E2
:104880008230B9F08330D9F48B8381EF8C833D8300
:1048900019C085E08B8381EF8C832F5F2D8312C03D
:1048A0008B8381EF8C8384E6489FA00111245D8374
:1048B00009C084E08B8381EF8C83ED8303C00E9469
:1048C000B81104C0CE0101960E94D5232996E2E0DA
:1048D0000C94102EA2E0B0E0E0E7F4E20C94E92D95
:1048E000182F762E2A8349830E9468286B017C0149
:1048F0008091DB048090C6049090C704A090C80407
:10490000B090C9042A8149818823C1F0D701C6012A
:1049100088199909AA09BB094C015D0191EE891614
:104920009EE29906A104B10420F1241708F4422F55
:10493000202F672D812F0E94272413C0D701C60185
:1049400088199909AA09BB094C015D0191E38916EF
:1049500095E79906A104B10460F0672D812F0E94AC
:104960007D23C092C604D092C704E092C804F0929E
:10497000C9042296EDE00C94052EA2E2B0E0E3EC2F
:10498000F4E20C94EA2D8CE00E94980981110DC08C
:104990006BE173E080EE95E00E94372A2C9A80E06C
:1049A0000E947D0A0E94580B2C9880EE95E00E9490
:1049B0004B2B892B01F180EE95E00E94782B909192
:1049C000A704992319F00E94BB13EFCF40913E0436
:1049D00050E09A012F5F3F4F2F71332760913F04C2
:1049E00070E02617370709F3FA01E75BFB4F808376
:1049F00020933E04DACF80917105843009F086C09F
:104A00000E946828611571058105910549F0609340
:104A1000B5047093B6048093B7049093B8040CC0A7
:104A200081E090E0A0E0B0E08093B5049093B604FC
:104A3000A093B704B093B8048091AB049091AC04F8
:104A400081609093AC048093AB0483E08093710504
:104A50008FE70E94760909E614E00E948909F801AF
:104A600081938F01F4E002371F07B9F72091720498
:104A700080916904982F922796FF3BC090E492277B
:104A800090937204982F98739833F1F410E0212FCB
:104A900030E080916904877090E0821793074CF1B1
:104AA0001F5F20919C05812F90E0FC01E759FB4F8F
:104AB00024FF04C080810E949A11E9CF608180EEBA
:104AC00095E00E94A52BE3CF8F7399F480916A043F
:104AD0008093B40480916B048093B20480916C0441
:104AE0008093B10480916F0490E09093AA04809326
:104AF000A90480913D04813019F482E080933D0443
:104B000080913D04833011F410923D040E94682886
:104B10006B017C018091AD049091AE04A091AF0433
:104B2000B091B0040097A105B105C9F0A7019601A5
:104B3000281B390B4A0B5B0BDA01C901883B9B40F0
:104B4000A105B10560F00E94C7098093B3041092DB
:104B5000AD041092AE041092AF041092B004809194
:104B6000B9049091BA04A091BB04B091BC04460171
:104B70005701881A990AAA0ABB0A84E795E00E949D
:104B8000F40786169706A806B90608F4A8C0C092CE
:104B9000B904D092BA04E092BB04F092BC040E9423
:104BA00057068091A8048830A0F08091BD059091AF
:104BB000BE05A091BF05B091C0055CE1B695A79573
:104BC000979587955A95D1F7892B8A2B8B2B09F0CE
:104BD0009EC18091A8048F5F8093A8048091B50442
:104BE0009091B604A091B704B091B8040097A105C4
:104BF000B105F1F0C81AD90AEA0AFB0A84E795E080
:104C00000E94F4076C157D058E059F0508F006C10E
:104C10008091BD0584FD04C080ED97E00E94A80747
:104C20001092B5041092B6041092B7041092B80412
:104C300090917204907C9093720450913E04809104
:104C40003F0420913D04581709F405C1223009F0B2
:104C500002C1905890937204E0919C05E770F0E0D7
:104C6000E758FC4F6081693008F0DDC0615040E0DA
:104C70004613DBC080933F0487E3840F9091720456
:104C8000892B809372044093400483E080933D0419
:104C90002B9A809181059091C304911129C10E94A2
:104CA000780A8091C4040E94B109E0919C05E770E4
:104CB000F0E0E758FC4F608182E794E00E94930B9C
:104CC000E091C404EF5FE093C404E83109F41CC12F
:104CD000F0E0EC58FA4F8785882309F415C10E944B
:104CE000020C813069F580919C05887149F18091B1
:104CF000AB049091AC04880F991F9093AC048093FF
:104D0000AB0483E0809371050E94580B0E946828D1
:104D10006093AD047093AE048093AF049093B0049D
:104D2000672B682B692B61F481E090E0A0E0B0E094
:104D30008093AD049093AE04A093AF04B093B004FD
:104D400080919C0584FF1FC08091AB049091AC04BE
:104D50008E7F0E942A09182F6091A9048091B404C3
:104D60000E94B113482F612F8091B30449A30E9480
:104D7000B1130091D205282F49A16091B10480910F
:104D8000B2040E946A242B988091C1048130C1F042
:104D900018F08230B1F1C8C08AE00E948129892BC5
:104DA00009F0C2C081E08093C1040E945C28609336
:104DB000BD047093BE048093BF049093C004B4C03C
:104DC0008AE00E948129892B31F50E945C28C090DD
:104DD000BD04D090BE04E090BF04F090C0046C19F4
:104DE0007D098E099F09693E73408105910508F48C
:104DF0009BC082E08093C10480ED97E00E94A807E9
:104E000093C08AE00E948129892B09F48DC080E03B
:104E100090E00E94A8071092C10486C080E090E054
:104E20000E94A80705CF68E022CF851709F422CF9A
:104E30004F5F242F30E090E0F901EE58FB4FDC018A
:104E4000A75BBB4F7C917083F901E05CFB4F7083E3
:104E500001968F710DCF2430B1F42091400481E48C
:104E600094E0A3E7B4E0FC013E2F381B321718F49E
:104E700031913D93F9CF87E3820F90917204892B92
:104E80008093720402CF8091C104823051F491600A
:104E9000909372042C9A8E010F5F1F4FF12CB80172
:104EA00010C02C9880913D04811103C081E0809353
:104EB0003D0480913D04833071F784E080933D048C
:104EC000EACF8F2D69A37AA30E94B315F8018193CD
:104ED00091938F01F39469A17AA1F0E1FF12F1CFD0
:104EE00080919C0543E754E087700E947908D0CEFA
:104EF000882309F4D4CE2091C20431E0320F3093DC
:104F0000C2042913CCCE0CC01092C404E8CE809108
:104F1000A804883009F42C9A89E08093A804DFCE95
:104F20001092C2048150BBCEA296ECE00C94062EE7
:104F30008230E8F4E82FF0E0EE0FFF1FED52FA4F59
:104F400071836083813041F0809169008C7F842B74
:104F500080936900E89A089580916900440F551F75
:104F6000440F551F837F842B80936900E99A08952D
:104F70001F920F920FB60F9211242F933F934F93CE
:104F80005F936F937F938F939F93AF93BF93EF93B1
:104F9000FF938091D3059091D405892B29F0E0915E
:104FA000D305F091D4050995FF91EF91BF91AF9191
:104FB0009F918F917F916F915F914F913F912F9131
:104FC0000F900FBE0F901F9018951F920F920FB663
:104FD0000F9211242F933F934F935F936F937F937F
:104FE0008F939F93AF93BF93EF93FF938091D505DA
:104FF0009091D605892B29F0E091D505F091D60541
:105000000995FF91EF91BF91AF919F918F917F9102
:105010006F915F914F913F912F910F900FBE0F9025
:105020001F9018951F920F920FB60F9211242F9375
:105030003F938F939F93AF93BF938091D8059091A7
:10504000D905A091DA05B091DB053091D70523E0B1
:10505000230F2D3720F40196A11DB11D05C026E8B0
:10506000230F0296A11DB11D2093D7058093D8056B
:105070009093D905A093DA05B093DB058091DC0508
:105080009091DD05A091DE05B091DF050196A11D8F
:10509000B11D8093DC059093DD05A093DE05B093F0
:1050A000DF05BF91AF919F918F913F912F910F900D
:1050B0000FBE0F901F9018952FB7F8946091D805E8
:1050C0007091D9058091DA059091DB052FBF089585
:1050D0003FB7F8948091DC059091DD05A091DE0545
:1050E000B091DF0526B5A89B05C02F3F19F00196AA
:1050F000A11DB11D3FBF6627782F892F9A2F620F00
:10510000711D811D911D42E0660F771F881F991F39
:105110004A95D1F70895CF92DF92EF92FF92CF9305
:10512000DF936B017C010E946828EB01C114D1045C
:10513000E104F10479F00E9468286C1B7D0B683E45
:105140007340A0F381E0C81AD108E108F108C85102
:10515000DC4FECCFDF91CF91FF90EF90DF90CF90BD
:105160000895789484B5826084BD84B5816084BDDF
:1051700085B5826085BD85B5816085BDEEE6F0E0D0
:10518000808181608083E1E8F0E01082808182602C
:105190008083808181608083E0E8F0E080818160AD
:1051A0008083E1EBF0E0808184608083E0EBF0E0DD
:1051B000808181608083EAE7F0E080818460808381
:1051C000808182608083808181608083808180682B
:1051D00080831092C1000895833081F028F48130DB
:1051E00099F08230A1F008958630A9F08730B9F0A7
:1051F0008430D1F4809180008F7D03C08091800045
:105200008F7780938000089584B58F7702C084B52E
:105210008F7D84BD08958091B0008F7703C0809109
:10522000B0008F7D8093B0000895CF93DF9390E01E
:10523000FC01ED50F44F2491FC01E95FF34F8491A0
:10524000882349F190E0880F991FFC01E15DF34F3D
:10525000A591B4918B5D934FFC01C591D4919FB7FB
:10526000611108C0F8948C91209582238C938881D9
:1052700082230AC0623051F4F8948C91322F309519
:1052800083238C938881822B888304C0F8948C912B
:10529000822B8C939FBFDF91CF910895A1E0B0E066
:1052A000E4E5F9E20C94F22D282F30E0F901E15207
:1052B000F44F8491F901ED50F44F1491F901E95F35
:1052C000F34F04910023C9F0882321F069830E94E1
:1052D000EC286981E02FF0E0EE0FFF1FEB5DF34F4C
:1052E000A591B4919FB7F8948C91611103C010956A
:1052F000812301C0812B8C939FBF2196E4E00C9405
:105300000E2ECF93DF93282F30E0F901E152F44FB6
:105310008491F901ED50F44FD491F901E95FF34F15
:10532000C491CC2391F081110E94EC28EC2FF0E085
:10533000EE0FFF1FE55EF34FA591B4912C912D2345
:1053400081E090E021F480E002C080E090E0DF9115
:10535000CF910895A0E0B0E0E0EBF9E20C94EE2DDF
:105360006C017A01EB01E60EF71E00E010E0CE15AD
:10537000DF0561F06991D601ED91FC910190F0811A
:10538000E02DC6010995080F191FF1CFC801CDB74F
:10539000DEB7E8E00C940A2E6115710589F0DB0197
:1053A0000D900020E9F7AD0141505109461B570B04
:1053B000DC01ED91FC910280F381E02D09950895C7
:1053C00080E090E00895EF92FF920F931F93CF93A8
:1053D000DF938C01FB01C0E0D0E064917F018FEF8F
:1053E000E81AF80A662361F0D801ED91FC9101906A
:1053F000F081E02DC8010995C80FD91FF701EDCF45
:10540000CE01CDB7DEB7E6E00C940C2E0E94CC297D
:105410000895DC01ED91FC910190F081E02D09955A
:1054200008950F931F93CF93DF93EC016DE00E94DB
:10543000092A8C016AE0CE010E94092A800F911F7F
:10544000DF91CF911F910F9108950F931F93CF93E9
:10545000DF93EC010E94E3298C01CE010E94112A06
:10546000800F911FDF91CF911F910F9108950F939E
:105470001F93CF93DF93EC010E94CC298C01CE01C6
:105480000E94112A800F911FDF91CF911F910F91E0
:1054900008950F931F93CF93DF93EC010E94092A85
:1054A0008C01CE010E94112A800F911FDF91CF91B4
:1054B0001F910F910895A1E2B0E0E1E6FAE20C94A9
:1054C000EA2D7C01C42EE52FCB01D22E19A221E0BA
:1054D0002D1510F02AE0D22E8E010F5D1F4F8D2C5E
:1054E000912CA12CB12C6C2D7E2FA50194010E9432
:1054F000A32D8C2DD29E80191124015011098A30C0
:1055000010F4805D01C0895CF801808321153105AC
:105510004105510521F0C22EE32FCA01E4CFB801A5
:10552000C7010E94CC29A196ECE00C94062EA0E0C5
:10553000B0E0EDE9FAE20C94EE2DEC016A017B019A
:105540002115310541F4E881F9810190F081E02DC8
:10555000642F09951DC02A303105A9F477FF12C0C8
:105560006DE20E94092A8C0144275527BA014C1983
:105570005D096E097F092AE0CE010E945B2A800F37
:10558000911F06C02AE0B701A601CE010E945B2A46
:10559000CDB7DEB7E8E00C940A2E9A01AB0166277E
:1055A00057FD6095762F0E94972A08950F931F93B9
:1055B000CF93DF93EC019A01AB01662757FD60950D
:1055C000762F0E94972A8C01CE010E94112A800F0B
:1055D000911FDF91CF911F910F91089521153105F2
:1055E00049F4DC01ED91FC910190F081E02D642FF4
:1055F000099508950E945B2A08959A01462F50E06C
:1056000060E070E00E94EE2A08959A01AB0160E02C
:1056100070E00E94EE2A08950F931F93CF93DF93BB
:10562000EC010E94EE2A8C01CE010E94112A800F0B
:10563000911FDF91CF911F910F9108950F931F93A9
:10564000CF93DF93EC019A01AB0160E070E00E9420
:10565000EE2A8C01CE010E94112A800F911FDF914A
:10566000CF911F910F9108950F931F93CF93DF93C5
:10567000EC019A01462F50E060E070E00E94EE2AB3
:105680008C01CE010E94112A800F911FDF91CF91D2
:105690001F910F910895FC0124853585F901E05C87
:1056A000FF4F80819181F901EE5BFF4F20813181B5
:1056B000821B930B8F7399270895FC018485958530
:1056C000FC01E05CFF4F40815181FC01EE5BFF4F2C
:1056D000208131814217530741F00190F081E02D84
:1056E000E80FF91F808190E008958FEF9FEF0895F4
:1056F000FC0184859585FC01E05CFF4F4081518170
:10570000FC01EE5BFF4F208131814217530779F096
:10571000A081B181A80FB91F8C91208131812F5FA9
:105720003F4F2F7333273183208390E008958FEF0D
:105730009FEF0895FC0181A1882329F0A489B589F0
:105740008C9186FFFBCF11A20895CF93DF93FC01CC
:1057500026853785D901A05CBF4F8D919C9111970B
:1057600001968F739927E901CE5BDF4F48815981FC
:1057700084179507D9F30D90BC91A02DA20FB31FEC
:105780006C93A685B785A05CBF4F11969C938E93B2
:10579000A689B7892C9181E090E0078C02C0880F20
:1057A000991F0A94E2F7282B2C9381E081A30488A7
:1057B000F589E02D80818064808381E090E0DF9135
:1057C000CF91089508951F920F920FB60F92112452
:1057D0002F933F934F938F939F93EF93FF938091DA
:1057E000C00082FD1CC04091C60080918606909149
:1057F000870601968F739927209188063091890634
:105800008217930771F0E0918606F0918706EA5BB4
:10581000F94F4083909387068093860602C080915B
:10582000C600FF91EF919F918F914F913F912F91E2
:105830000F900FBE0F901F90189580EE95E00E947C
:105840004B2B892B11F00E94E22B08951F920F928F
:105850000FB60F9211242F933F938F939F93EF9343
:10586000FF93209142063091430680914406909127
:1058700045062817390731F48091C1008F7D809348
:10588000C10014C0E0914406F0914506EE5FF94F67
:105890002081809144069091450601968F73992747
:1058A00090934506809344062093C600FF91EF91A4
:1058B0009F918F913F912F910F900FBE0F901F904E
:1058C0001895A0E0B0E0E7E6FCE20C94EA2DFC01BC
:1058D0001382128288EE93E0A0E0B0E08483958387
:1058E000A683B7838BEB93E091838083758764876E
:1058F00057874687318B208B138B028BF58AE48A7E
:10590000D78AC68AB18EA08E938E828E8F85848F21
:105910008889858F8989868F8A89878F8B8980A3DB
:10592000ECE00C94062ECF92DF92EF92FF92CF9391
:10593000DF93EC016A017B01411581EE5807610597
:105940007105F9F0EC89FD8981E090E008A002C0C2
:10595000880F991F0A94E2F7808360E079E08DE375
:1059600090E0A70196010E94A32D21503109410921
:1059700051095695479537952795211580E13807A8
:1059800098F0EC89FD89108260E874E88EE190E07F
:10599000A70196010E94A32D215031094109510907
:1059A0005695479537952795E889F9893083EA898F
:1059B000FB89208319A2EE89FF89408181E090E074
:1059C0009C010C8C02C0220F331F0A94E2F7422B79
:1059D0004083EE89FF8940819C010D8C02C0220F1B
:1059E000331F0A94E2F7422B4083EE89FF894081FE
:1059F0009C010E8C02C0220F331F0A94E2F7422B47
:105A00004083EE89FF8920810F8C02C0880F991F87
:105A10000A94E2F7809582238083DF91CF91FF90F3
:105A2000EF90DF90CF9008958F929F92AF92BF92A8
:105A3000CF92DF92EF92FF920F931F9381E08F93AB
:105A400085E08F9387E08F9383E08F9384E08F933B
:105A5000E6EC8E2E912CF2ECAF2EB12CA1ECCA2EDE
:105A6000D12CB0ECEB2EF12C04EC10E025EC30E066
:105A700042E056E066E476E080EE95E00E94612C1C
:105A80000F900F900F900F900F901F910F91FF901C
:105A9000EF90DF90CF90BF90AF909F908F90089540
:105AA0000E94B1280E942122CDE1DCE20E94BD24A7
:105AB0002097E1F30E941D2CF9CFA29FB001B39F64
:105AC000C001A39F700D811D1124911DB29F700D07
:105AD000811D1124911D08950E945D2DA59F900D9B
:105AE000B49F900DA49F800D911D11240895B7FFC0
:105AF0000C946C2D0E946C2D821B930B0895DB017E
:105B00008F939F930E946C2DBF91AF91A29F800DA8
:105B1000911DA39F900DB29F900D1124089597FBA6
:105B2000072E16F4009407D077FD09D00E94212E8D
:105B300007FC05D03EF4909581959F4F0895709590
:105B400061957F4F0895A1E21A2EAA1BBB1BFD0190
:105B50000DC0AA1FBB1FEE1FFF1FA217B307E4074C
:105B6000F50720F0A21BB30BE40BF50B661F771FA4
:105B7000881F991F1A9469F7609570958095909584
:105B80009B01AC01BD01CF010895052E97FB1EF4CA
:105B900000940E94DC2D57FD07D00E94A32D07FC26
:105BA00003D04EF40C94DC2D509540953095219502
:105BB0003F4F4F4F5F4F0895909580957095619539
:105BC0007F4F8F4F9F4F08952F923F924F925F923A
:105BD0006F927F928F929F92AF92BF92CF92DF92FD
:105BE000EF92FF920F931F93CF93DF93CDB7DEB762
:105BF000CA1BDB0B0FB6F894DEBF0FBECDBF0994F6
:105C00002A88398848885F846E847D848C849B844C
:105C1000AA84B984C884DF80EE80FD800C811B815A
:105C2000AA81B981CE0FD11D0FB6F894DEBF0FBE89
:105C3000CDBFED010895EE0FFF1F0590F491E02D0B
:105C40000994AA1BBB1B51E107C0AA1FBB1FA617C3
:105C5000B70710F0A61BB70B881F991F5A95A9F715
:105C600080959095BC01CD0108958F929F92AF923F
:105C7000BF92CF92DF92EF92FF92CF93DF93EC012E
:105C8000688179818A819B81611571058105910502
:105C900021F464E279ED8BE597E02DE133EF41E00B
:105CA00050E00E94C52D49015A019B01AC01A7EAB1
:105CB000B1E40E946C2D6B017C01ACEEB4EFA50148
:105CC00094010E947A2DC60ED71EE81EF91EF7FE1B
:105CD00006C081E0C81AD108E10880E8F80AC88245
:105CE000D982EA82FB82C701B6019F77DF91CF910B
:105CF000FF90EF90DF90CF90BF90AF909F908F90EC
:105D000008950E94352E089586E091E00E94352E78
:105D100008956093060170930701809308019093A2
:105D2000090108952F923F925F926F927F928F9216
:105D30009F92AF92BF92CF92DF92EF92FF920F931A
:105D40001F93CF93DF938B01EA016115710521F059
:105D5000DB018C9311969C93209739F09E01225081
:105D600031092332310508F0D8C07C016701BFEF4B
:105D7000CB1ADB0A5601F7016080862D90E00E9465
:105D8000C42F892B11F07601F1CFFDE26F120AC00A
:105D9000570182E0A80EB11CD70111966C907724B0
:105DA00073940BC0BBE26B1207C05701E2E0AE0E6A
:105DB000B11CD70111966C90712CCE018F7E892B6E
:105DC00089F4B0E36B1237C0F50180818F7D88358F
:105DD000D1F46180F2E0AF0EB11C872D8260782E85
:105DE000C0E1D0E0CA30D10551F1C031D10521F078
:105DF000C830D10599F409C0CC24CA94DC2CEC2C11
:105E0000AFE0FA2E22C0209769F7C8E0D0E0CC249A
:105E1000CA94DC2CEC2CFFE1FF2E17C06FEF7FEF54
:105E2000CB019E01442737FD4095542F0E94A32D9E
:105E300069017A010AC02097A9F6CAE0D0E0E9E931
:105E4000CE2EDC2CEC2CE9E1FE2EF50160E020E00A
:105E500030E0A9014E01AA2497FCA094BA2C1F019E
:105E600070ED572E560CA9E0A51570F48FEB860D3A
:105E70008A3118F499EC592E06C08FE9860D8A31C3
:105E800048F589EA582E560C852D90E08C179D0711
:105E90000CF56F3FD9F0C216D306E406F50698F06C
:105EA000C501B4010E947F2D9B01AC01852D90E0BE
:105EB000A0E0B0E0280F391F4A1F5B1F28173907E1
:105EC0004A075B0710F46FEF01C061E03196D10122
:105ED0006C90C5CF0115110551F0662311F0319773
:105EE00003C071FE04C03297D801ED93FC9370FE9D
:105EF00007C050954095309521953F4F4F4F5F4FCC
:105F000067FF10C082E290E090938B0680938A0630
:105F10006FEF7FEF8FEF9FEF07C060E070E080E0F2
:105F200090E002C0B901CA01DF91CF911F910F919A
:105F3000FF90EF90DF90CF90BF90AF909F908F90A9
:105F40007F906F905F903F902F900895FC0188277D
:105F50009927E89421912032E9F3293010F02E306E
:105F6000C8F32B3241F02D3239F4689404C00E94FA
:105F7000F82F820F911D219120532A30C0F31EF477
:105F8000909581959F4F0895911150C0803219F0DE
:105F900089508550D0F7089548EC53E00E94D12FE6
:105FA0000895FA01A191B081009719F41097E1F0DA
:105FB000CD01DC01CD010D90002011F4C00113C012
:105FC000FB012191222319F02015D9F7F3CFFB0112
:105FD0002191201519F41E92119606C02223C1F7B3
:105FE0000D900020A1F7D001FA01A193B08308958C
:105FF0007AE0979F902D879F802D910D1124089511
:10600000F999FECF92BD81BDF89A992780B5089580
:10601000262FF999FECF1FBA92BD81BD20BD0FB6C4
:10602000F894FA9AF99A0FBE01960895992788274D
:066030000895F894FFCF73
:1060360000008C06200001000000FF0002000200A4
:10604600020002000200020002000200020002003A
:106056000200020002000200020002802500000584
:10606600400AA1204EA50020244EA52C2330C012A4
:1060760000001A400AA1204EA5001B1E27522C2301
:10608600308025000005400AA1204EA50020244EA0
:10609600A52C2330004B000006400AD0009D490085
:1060A6007B289D492C233000E1000005400A45016C
:1060B600D7DC03B81E0EBF00232E48E801008A4035
:1060C6000A6001555502AD1E20000023C854582011
:1060D60074696D656F75742100596573004E6F00A4
:1060E6002C00386368004E2F41002C205B005D2099
:1060F60028002900486F70206368616E6E656C2009
:106106000020402000456E746572696E67206164E8
:10611600617074697665206368616E6E656C207364
:10612600656C656374696F6E2C207069636B696E4C
:10613600673A007363616E6E6572206D6F64650009
:106146004E4F5420454E41424C45440053656E64C3
:10615600696E672073657474696E677320746F2047
:1061660052580A00526573657474696E67207365C8
:106176007474696E6773206F6E2052580A0041620C
:106186006F727465642065646974730A00696E765B
:10619600616C69642073656C656374696F6E000D6C
:1061A6000A496E76616C696420696E707574202D7B
:1061B60020646973636172646564210700536574C2
:1061C60074696E677320736176656420746F204509
:1061D6004550524F4D0A00526576657274656420CB
:1061E60073657474696E67732066726F6D204545BA
:1061F60050524F4D0A004C6F6164656420666163BE
:10620600746F72792064656661756C74730A004BED
:10621600657920616E64206368616E6E656C7320BB
:1062260072616E646F6D697A65640A004F70656E9F
:106236004C52536E67205458207374617274696EA1
:10624600672000206F6E20485720006D6F64756CC4
:1062560065206C6F636B65643F00342B3400380037
:10626600382B340031320031322B340031360050B5
:10627600504D0052535349005344410053434C0080
:10628600525844005458440041494E004C4245453A
:10629600500053504B54524D0053425553005355E2
:1062A6004D44004C4C494E440000070B0C10111590
:1062B60000B6012A032E033003340337033C03B62A
:1062C600013F03430348034C035003540358035C44
:1062D60003620369036E0373038C028C028C028CC7
:1062E60002160A1322312900000000A52BAA294B09
:0862F6002B782B5D2B9A2B0085
:107E00000F92CDB7DEB7112484B714BE81FFF1D035
:107E100082E08093C00088E18093C10086E0809377
:107E2000C20080E18093C4008EE0CDD088249924E4
:107E3000CC24C394F5E0DF2EE1E1EE2E73E0F72EC3
:107E4000B6D0082F813479F4B2D08983C2D0898129
:107E5000823811F481E005C0813811F485E001C059
:107E600083E09ED09AC0823411F484E103C085344B
:107E700019F485E0B6D091C0853561F498D0082F0B
:107E800010E095D090E0982E8824802A912A880CC2
:107E9000991C82C0863521F484E0A3D080E0E1CF34
:107EA000843609F04CC083D082D0A82E80D0B82E62
:107EB00000E011E07CD0F80181938F01AE16D1F77C
:107EC00088D0FB2DF53489F4E0E0F1E00BC0F9999E
:107ED000FECF92BC81BC0894811C911C819180BD15
:107EE000FA9AF99AEA1598F358C08B2D863409F05E
:107EF00054C0F401F7BEE89507B600FCFDCFF401CD
:107F0000A0E0B1E02C9130E011968C91119790E0B7
:107F1000982F8827822B932B12960C01C7BEE895C9
:107F20001124329681E0A038B80761F7F401D7BE7A
:107F3000E89507B600FCFDCFE7BEE8952EC0843774
:107F4000F1F435D034D0182F32D0B82E42D0FB2DDA
:107F5000F63421F4F40105914F010CC0FB2DF534EA
:107F600049F4F999FECF92BC81BC0894811C911C04
:107F7000F89A00B5802F14D0115049F70EC08537FC
:107F800039F427D08EE10CD085E90AD08FE069CF93
:107F9000813511F488E017D01CD080E101D050CF9A
:107FA0009091C00095FFFCCF8093C600089580910A
:107FB000C00087FFFCCF8091C00084FD01C0A89560
:107FC0008091C6000895E0E6F0E098E19083808318
:107FD0000895EDDF803219F088E0F5DFFFCF84E10E
:107FE000DFCF1F93182FE3DF1150E9F7F2DF1F9166
:0E7FF0000895282E80E0E7DFEE27FF27099492
:027FFE0001057B
:0400000300007E007B
:00000001FF
